:10007C0001501040202F212BD9F708950EBBE09A88
:10008C000DB308950EBB4DBBE29AE19AE199FECFF8
:10009C00089501501040202F212BD9F703E007B908
:1000AC00089530D1B99ABB9A379A369A359A3398C3
:1000BC00329A3198309801E007B908E900BF00E89E
:1000CC0008B9C39A0BE0DADF402E552400E1D6DFE5
:1000DC001127400E511E542C4424A8ECAA2351F095
:1000EC0085B19927982F8827079604E610E0C0DF82
:1000FC00AA95F4CF06E900BF00EC0EBD08EC1FEA90
:10010C00B7DF002700BF07E900BF00EC0EBD08EC0D
:10011C001FEAAEDF002700BF08E900BF00EC0EBDF0
:10012C0008EC1FEAA5DF002700BF06E900BF00ECC2
:10013C000EBD08EC1FEA9CDF002700BFC39800E14E
:10014C009DDF0395402F00E19DDFE6E6F0E0C895CA
:10015C000DE4001609F0B5CF25B13327322F222735
:10016C0004B11127202B312B280F391F822F932FED
:10017C0004E110E07DDF082F192F4CE050E09AD0FD
:10018C00802F912F0296E3E6F0E0C89507E4001665
:10019C0009F097CF0EE110E07CDF08E116EF68DF85
:1001AC0008E116EF65DF08E116EF62DFBB27662476
:1001BC00772401E010E0012B09F477C0E4E6F0E0CD
:1001CC00C8950EE4001609F07CCF88279927AA273A
:1001DC00A03488F425B13327322F222704B11127FC
:1001EC00202B312B280F391F822F932F0EE110E07B
:1001FC003FDFA395EDCFBB2319F4482E592EB1E068
:10020C008415950528F4242D352D281B390B02C097
:10021C0022273327213500E03007B8F0939405E00E
:10022C00901660F0992466247724C39A06E900BFDF
:10023C00369527953695279520952EBD8824A39421
:10024C00AA2069F4482E592E0AC0C398002700BF73
:10025C00AA2499248394882011F4482E592E0FEF48
:10026C00601A700A09E0601602E57006B0F0BB2750
:10027C0066247724AA27A33080F4C39A07E900BF29
:10028C0000EE0EBD00E61AEEF3DEC398002700BFA9
:10029C0000E61AEEEDDEA395EECFEBE6F0E0C895A6
:0E02AC0006E5001609F019CF84CFEBE03CC048
:1000620020474E4F4D2D4D5F41564F5F323031305C
:090072002A20000073656E640091
:020000000FC02F
:10001C0000EC05BFC0E800E903500DBF49D1002337
:10002C0009F417D0E0E6F0E000E060D1E2E6F0E0A1
:10003C0000E640E04FD1E0E6F0E000E057D1E2E628
:10004C00F0E000E640E046D1E2E6F0E000E640E019
:06005C0041D127D02CC1A8
:0202BA00FFCF74
:0402BC0001E00895C0
:1002C000002411240030010741F01695079510F421
:1002D000040E151E440F551FF5CF002D112D089546
:1002E000BF93AF93A02F03C0C89531960D92415094
:0802F000D8F7AF91BF9108950A
:0C02F800002401C001920150E8F70895B5
:020304000000F7
:10030600FA92EA92DA92CA92BA92AA929A928A9247
:100316007A926A925A924A92BA93AA939A938A9333
:02032600089538
:10032800FF84EE84DD84CC84BB84AA849984888489
:100338007F806E805D804C80BB81AA819981888195
:0E034800F0E00FB6F894CE0FDF1F0FBE089541
:00000001FF
